:020000040000FA
:0400000047EF09F0CD
:08000800056ED8CF06F0E0CF31
:1000100007F00001E9CF0DF0EACF08F0E1CF09F0D9
:10002000E2CF0AF0D9CF0BF0DACF0CF0F3CF14F017
:10003000F4CF15F0FACF16F000C00FF001C010F0A9
:1000400002C011F003C012F004C013F09DA02CEF09
:1000500000F09EB098EF01F09DAA32EF00F09EBA3A
:1000600070EF00F00FC000F010C001F011C002F0FE
:1000700012C003F013C004F00E8E0DC0E9FF08C0DB
:10008000EAFF09C0E1FF0AC0E2FF0BC0D9FF0CC0C4
:10009000DAFF14C0F3FF15C0F4FF16C0FAFF0550D5
:1000A00007C0E0FF06C0D8FF1000F2CF0EF0F29EAE
:1000B000F76AC40FF66E000EF7220900F5500EBE67
:1000C000F28E1200312E312E33000101306B2F6B76
:1000D000AB98030E006E002EFED7AB880001000C1B
:1000E000CE500101B36FCFCFB4F19EAAFED7AECFF1
:1000F000F5F12F5303E10001E8DF0101F55102089A
:1001000001E1306B036A30512F0FE96E000E0320BE
:10011000EA6EF5C1EFFF302B3051800804E1000199
:10012000D4DF1AD00101F551030813E130C131F1D8
:10013000EA6AAF0EE96EE26A2F0EE16E3151016E8E
:1001400004E0E6CFEEFF012EFCD70001BEDF04D0B5
:100150000101050E2F6F00019E9A32EF00F0036A35
:100160000101B251320FE96E010E0320EA6EFDC1AA
:10017000EFFFB22B0001000C0101FCBF11D00F0EEC
:10018000006EFB3900160A0E005C03E2300E0026FA
:1001900002D0FC51002600C0FDF10001E0DF0101AA
:1001A0000F0EFB170A0EFB5D02E2300E02D0FC9F21
:1001B000FC51FB27FBC1FDF10001D1DF000C010167
:1001C000B26B020EFD6F0001CADFF9C1FBF1370E01
:1001D0000101FC6F0001D0DFFAC1FBF1370E010114
:1001E000FC6F0001C9DF000C8B940201046B045109
:1001F0000F082AE3000B006E0151800B036E0050C4
:10020000031002E08B8001D08B90000B006E035135
:10021000800B036E0050031002E08B8201D08B92A2
:10022000100E006E002EFED700008B84100E006EA4
:10023000002EFED700008B94D89000370137D8905D
:1002400002370337042BD3D700014EEF01F0FCC176
:1002500000F20101FD510F0B0201016FFCC1FCF125
:100260000201015170090101FD6FFEC100F201019F
:10027000FF510F0B0201016FFEC1FEF1020101519E
:1002800070090101FF6F8B96FDC101F2FCC100F204
:10029000FFC103F2FEC102F20001A6D78B8604EF74
:1002A00002F004000101FC519EA8FED7AD6EACB275
:1002B00002D00400FCD70001000C0101B251040877
:1002C00002E3B26B33D0F96B010EFA6FB251FA5DF3
:1002D0000BE2036AFA51320FE96E010E0320EA6E57
:1002E000EF50F927FA2BF2D7F91FF9C1FBF1370EBE
:1002F000FC6F000141DF030E0101FD6F00012FDFE4
:100300000101FA6BB251FA5D10E2036AFA51320F41
:10031000E96E010E0320EA6EEFCFFBF1FBC1FCF1A9
:100320000001BFDF0101FA2BEDD7B26B0001000C19
:100330000B0ECF6EDB0ECE6E1D2A0101CA2B2C2AAE
:100340001D5009080FE21D6A1E2A1E503C0809E1D3
:100350001E6A1F2A1F503C0804E11F6A202AD8B4D5
:10036000212A22802D502C5C53E32B5251E022A2F3
:100370004DD022B44BD0050EF96F080EFA6F000174
:100380001EDF0101BDC1F6F1BCC1F5F1BFC1F8F13D
:10039000BEC1F7F1F8C1FBF1370EFC6F0001ECDED6
:1003A000F7C1FBF1370E0101FC6F0001E5DEF6C17C
:1003B000FBF1370E0101FC6F0001DEDEF5C1FBF140
:1003C000370E0101FC6F0001D7DE036A0101BF3166
:1003D000026EBE31016EBD31006E0232013200325A
:1003E0000232013200320232013200320F0E0216A6
:1003F00001C0FBF100C0FAF101C0FDF100C0FCF149
:10040000FF6BFE6B000123D758DF01012C6A2B6ABA
:100410002F5301E02F07B65302E0B60704D022B4F1
:1004200002D08C908C929E90000132EF00F001017E
:10043000EF6BEF510E0820E3D10EEF25016E010E98
:10044000036ED8B0032A0150E96E03C0EAFF020E22
:10045000EF25F26F210EF36FD8B0F32BF2CFF4F14A
:10046000F29EF2C1A9FFA69CA69EA680A850F4BF4A
:10047000F28EEF6EEF2BDDD7DF2D11D0D0C1EAFF6A
:10048000CFC1E9FF010EE26ED10EE16E0F0E016EDB
:10049000E6CFEEFF012EFCD7010E016E02D0000E5A
:1004A000016E000176EF09F0010EEA6EE30EE96ECF
:1004B000EF500DE0060E016E006A002EFED7012EF1
:1004C000FBD77B0E006E002EFED7EF2EF3D7000C6D
:1004D00081B005D08C948C86010E016E04D08C9670
:1004E0008C94000E016E000C0101D76BD76AD66A9E
:1004F0000001EEDF01521EE0EBDF015208E10101D5
:10050000D72BD751050801E215D003D00001010116
:10051000D76BD650D56FD7CFD6F1D651D45D0AE37D
:10052000D8B402D00001E8D7D351D55DD8B002D0FD
:100530000001E2D70101D76B0001CADF01521EE1C1
:10054000C7DF015208E00101D72BD751010801E2B2
:1005500015D003D000010101D76BD650D56FD7CF8E
:10056000D6F1D651D45D0AE3D8B402D00001E8D761
:10057000D351D55DD8B002D00001E2D70101D651E8
:10058000D45D1CE303E1D351D55D18E2D76AD66A86
:100590001C6A1B6A1C50D45D11E303E1D3511B5C40
:1005A0000DE2000195DF015203E1010E016E08D05A
:1005B000D6501B6ED7CF1CF00101ECD7000E016E98
:1005C0000001000C0101D185D1912E6AD06B9D9064
:1005D0000B0ED46FB80ED36F000186DF015211E00D
:1005E0001C5000080AE2FF0A03E11B505E0805E206
:1005F000010E0101D26F03D000010101D26B03D0C3
:1006000000010101D181CB6BD1B117D00B0ED46F9A
:10061000B80ED36F000168DF01520DE01C500008D6
:1006200009E2FF0A03E11B505E0804E2010E01012A
:10063000CB6F000103D00101D18100010101D1B1D3
:1006400017D00B0ED46FB80ED36F00014DDF0152DF
:100650000DE01C50000809E2FF0A03E11B505E0890
:1006600004E2020E0101CB27000103D00101D18178
:1006700000010101D1B15CD0CF6BCF51060858E326
:10068000D1B156D0036ACF51230FE96E000E03207B
:10069000EA6EEF6AD06BD05107083AE3D1B138D097
:1006A0000B0ED46FB80ED36F00011EDF01520EE1A6
:1006B0000101D0510608D8B002D0000107D0CF51B7
:1006C0000508D8B002D0000101D0D1810101D1B11B
:1006D0001DD01C5000081AE2FF0A03E11B505E08FF
:1006E00015E2036ACF51230F016E000E032201C0F1
:1006F000E9FF03C0EAFF010E006ED051016E04E075
:10070000D8900036012EFCD70050EF12D02BC3D763
:10071000D1B10CD0CF51060809E0036ACF51230FA5
:10072000E96E000E0320EA6EEF502E26CF2BA5D7E0
:100730009D80D193D1B105D02E1E29502E5C01E1B0
:10074000D183D195D1A306D022A604D02450B85D80
:1007500001E1D185D1A506D02A50D25D01E1D19524
:10076000D2C12AF0D1A504D08C908C82050EB66F30
:10077000000ED1B5010E016E0001CFEF09F023C0CC
:10078000CCF1036A0101D76B036ACC51D725B96F4D
:100790000350CB21BA6FD591020ED66F036AD651A2
:1007A000230FE96E000E0320EA6EEF50F80809E10E
:1007B000036AD651230FE96E000E0320EA6EFF0E86
:1007C000EF6E036AD651230FE96E000E0320EA6E26
:1007D000EFCFBFF1010ED625036A230FE96E000E9D
:1007E0000320EA6EEFCFBEF1020ED625036A230F77
:1007F000E96E000E0320EA6EEFCFBDF1030ED625A1
:10080000036A230FE96E000E0320EA6EEFCFBCF1FE
:10081000BF5309E0BF3D01D006D07F0EBF6FFF0E72
:10082000BE6FBD6FBC6FBC3D09D0BD3D07D0BE3DA6
:1008300005D0BF517F0802E1D581228822A425D0AE
:10084000D5B123D0C3C1D2F1C2C1D1F1C1C1D0F160
:10085000C0C1CFF1BC51CF25006EBD51D021016E7A
:10086000BE51D121026EBF51D221D26F02C0D1F14F
:1008700001C0D0F100C0CFF1D2C1C3F1D1C1C2F1EA
:10088000D0C1C1F1CFC1C0F10AD0D5B108D0C0519B
:10089000BC5FC151BD5BC251BE5BC351BF5B22A4F3
:1008A00003D0D5B101D0C42B010E2B6E0001D3EFC4
:1008B00009F00101E8C1E9FFE9C1EAFFEFCFEBF17F
:1008C000010EE825016E000EE92101C0E9FFEA6E84
:1008D000EFCFECF1EB51390804E3300EEB5DEA6F3A
:1008E00004D0410EEB5D0A0FEA6FEA3BEC51390888
:1008F00004E3300EEC5DEA2704D0410EEC5D0A0FF4
:10090000EA27EAC101F00001000C0101315107089A
:1009100003E3000E016E40D00001AF5102080DE16B
:10092000010E0101315D036AAF0FE96E000E032075
:10093000EA6EEF50030805E00001000E016E0101B0
:100940002BD0CF6B010ED06F030E315DD05D0BE26B
:10095000036AD051AF0FE96E000E0320EA6EEF502C
:10096000CF27D02BF1D7CFC1D1F1D11F030E315DED
:10097000036AAF0FD36F000E0320D46FE96FD3C1AA
:10098000E8F1000196DF01500101D15D03E0000EA6
:10099000016E02D0010E016E0001E0EF09F0186A4D
:1009A000F2BE188EF29E0101F96BFA6B000107DCB2
:1009B00018BEF28E186AF2BE188EF29E7EDC18BE49
:1009C000F28E000C0101E437E333E433010EEA6EEA
:1009D000E70EE96E010EE26EE30EE16E040E016EAB
:1009E000E6CFEEFF012EFCD7EB6BEB51030819E3CA
:1009F000036AEB51E70FE96E010E0320EA6EEFCFB9
:100A0000ECF1186AF2BE188EF29EECC1FBF1370EC3
:100A1000FC6F0001BCEC00F018BEF28E0101EB2B64
:100A2000E4D70001000C0101E56BE5510E082AE353
:100A3000020EE525E66F210EE76FD8B0E72BE551F2
:100A4000E325016E000EE421036E01C0E9FFEA6EAA
:100A5000EFCFE8F1E6C1A9FFE8C1A8FFA69CA69EDA
:100A6000A684F2CF00F0F29E0F01550EA76EAA0EDB
:100A7000A76EA682A6B2FED7A6940050F21201017C
:100A8000E52BD3D70001000C22980101C36BC26B88
:100A9000C16BC06BC46B2284B56B000170EF08F0B2
:100AA0000101E96BB00EE86F000103DF01C0CFF177
:100AB0000101CF51020A000124E0170A24E01A0ABA
:100AC000D8B48CD01C0AD8B49ED1190AD8B4EDD1B0
:100AD000060AD8B420D2140AD8B453D2010AD8B422
:100AE00053D20F0AD8B453D20C0AD8B45ED2190A22
:100AF000D8B468D21E0AD8B467D2010AD8B48CD24E
:100B0000D9D24DDFEDD20101E96BB20EE86F0001E1
:100B1000D0DE015004084BE10101D26BD251010833
:100B200043E3036AD251D00F016E010E032201C0CC
:100B3000E3F103C0E4F1D890D235050F036AAF0F9B
:100B4000E66F000E0320E76FE96FE6C1E8F10001F0
:100B5000B0DEE4C1EAFFE3C1E9FF01C0EFFF01013C
:100B6000D2C1E3F1210E036AD251D00FE96E010E1A
:100B70000320EA6EEFCFE5F1D2C1A9FFE5C1A8FFDE
:100B8000A69CA69EA684F2CF00F0F29E0F01550E01
:100B9000A76EAA0EA76EA682A6B2FED7A694005094
:100BA000F2120101D22BBAD78BD016D00001186AED
:100BB000F2BE188EF29E010E0101F96FFA6B000170
:100BC000DFEC00F018BEF28E186AF2BE188EF29EAC
:100BD0005DEC01F018BEF28E000182D20101D26BF1
:100BE000D251010819E3036AD251D00FE96E010E08
:100BF0000320EA6ED251E56F210EE66FF2CFE7F1E6
:100C0000F29EE5C1A9FFA69CA69EA680A850E7BFBC
:100C1000F28EEF6ED22BE4D7D26BD25101080DE3E6
:100C2000036AD251D00FE96E010E0320EA6EEF3C49
:100C300001D001D002D0D22BF0D7D251020840E12E
:100C4000D26BD25101083CE3036AD251D00FE96E56
:100C5000010E0320EA6ED251080DF3CF00F0B4C1AB
:100C600003F0B3C102F0005205E0D8900332023223
:100C7000002EFBD702C0EFFFD2C1E3F1210E036AC1
:100C8000D251D00FE96E010E0320EA6EEFCFE5F1ED
:100C9000D2C1A9FFE5C1A8FFA69CA69EA684F2CF5B
:100CA00000F0F29E0F01550EA76EAA0EA76EA68247
:100CB000A6B2FED7A6940050F2120101D22BC1D7E2
:100CC00000016DDE186AF2BE188EF29E100E010150
:100CD000F96F180EFA6F0001DFEC00F018BEF28E0B
:100CE000186AF2BE188EF29E0C0E0101FB6F370ED1
:100CF000FC6F0001BCEC00F018BEF28E186AF2BE68
:100D0000188EF29E1D0E0101FB6F370EFC6F000165
:100D1000BCEC00F018BEF28E186AF2BE188EF29E7D
:100D2000020E0101FB6F370EFC6F0001BCEC00F0FE
:100D300018BEF28E0101D26B036AD251F2CFE3F1F9
:100D4000F29E000155EC00F00101E3BFF28E000AB3
:100D500019E0036AD251F2CFE3F1F29E000155ECA3
:100D600000F00101E3BFF28EE46F186AF2BE188E44
:100D7000F29EFD6F0001AFEC00F018BEF28E010193
:100D8000D22BDAD7D25105080EE3186AF2BE188EBC
:100D9000F29E200EFD6F0001AFEC00F018BEF28E47
:100DA0000101D22BEFD7D26BD251010819E3036AAC
:100DB000D251D00FE96E010E0320EA6EEFCFE3F1BE
:100DC000186AF2BE188EF29EE3C1FBF1370EFC6F7B
:100DD0000001BCEC00F018BEF28E0101D22BE4D76A
:100DE000C9C1E6F1C8C1E5F1C7C1E4F1C6C1E3F18B
:100DF0000001E8DD186AF2BE188EF29E5DEC01F08B
:100E000018BEF28E6DD1CBDD186AF2BE188EF29E3E
:100E1000140E0101F96F1C0EFA6F0001DFEC00F0F7
:100E200018BEF28E186AF2BE188EF29E010E0101F3
:100E3000FB6F370EFC6F0001BCEC00F018BEF28EA9
:100E4000186AF2BE188EF29E180E0101FB6F370E63
:100E5000FC6F0001BCEC00F018BEF28E400E0101E8
:100E6000E66FA10EE56F740EE46F790EE36F00017B
:100E7000A9DD400E0101E66FA10EE56F740EE46F6F
:100E8000790EE36F00019EDD0101E66BE56BE46B1B
:100E90007F0EE36F000196DD186AF2BE188EF29E97
:100EA0005DEC01F018BEF28E1BD179DD186AF2BE3E
:100EB000188EF29E0B0E0101F96F120EFA6F0001EF
:100EC000DFEC00F018BEF28E0101E66BE56B200E40
:100ED000E46F800EE36F000175DD0101E66BE56BE9
:100EE000E46BE36B00016EDD186AF2BE188EF29EB1
:100EF0000A0E0101FB6F370EFC6F0001BCEC00F025
:100F000018BEF28E186AF2BE188EF29E5DEC01F0E9
:100F100018BEF28EE5D043DD186AF2BE188EF29E3E
:100F2000080E0101F96F040EFA6F0001DFEC00F00A
:100F300018BEF28E020E0101E36F300E186AF2BE87
:100F4000188EF29EFD6F0001AFEC00F018BEF28E1D
:100F50000101E32FF2D7186AF2BE188EF29EB9C1D2
:100F6000FBF1370EFC6F0001BCEC00F018BEF28EF6
:100F7000186AF2BE188EF29E5DEC01F018BEF28E79
:100F8000AFD00DDD2282ACD00ADD2292A9D007DDE0
:100F9000F29CF29EF2BEFDD7320E0101E36F00011A
:100FA00054EC02F002EF3EF09BD0F9DC0101C36B80
:100FB000C26BC16BC06B010EE46FB70EE36F000133
:100FC00032DD8ED0ECDC60D5EADC0101E96BB80ED5
:100FD000E86F00016EDC01C0B7F10101E96BBA0EE8
:100FE000E86F000166DC01C0B8F10101C36BC26BA0
:100FF000C16BC06B010EC56F020EBB6F2286C96B41
:10100000C86B7A0EC76F880EC66F010EE46FB70EFD
:10101000E36F000108DD64D0C2DC186AF2BE188EEE
:10102000F29E1B0E0101F96F080EFA6F0001DFEC52
:1010300000F018BEF28E186AF2BE188EF29E010100
:10104000FB6B370EFC6F0001BCEC00F018BEF28E9B
:10105000186AF2BE188EF29E0101FB6B370EFC6F10
:101060000001BCEC00F018BEF28E186AF2BE188EB9
:10107000F29EB7C1FBF1370E0101FC6F0001BCEC21
:1010800000F018BEF28E186AF2BE188EF29EB8C139
:10109000FBF1370E0101FC6F0001BCEC00F018BE43
:1010A000F28E186AF2BE188EF29E5DEC01F018BE48
:1010B000F28E16D0186AF2BE188EF29E010E010151
:1010C000F96FFA6B0001DFEC00F018BEF28E186ABF
:1010D000F2BE188EF29E5DEC01F018BEF28E00D0CA
:1010E000E4EF09F00101D751DB19800BE16FD7AFB5
:1010F0000BD0D41FD51FD61FD71FD42BD8B4D52BB8
:10110000D8B4D62BD8B4D72BDBAF0BD0D81FD91F70
:10111000DA1FDB1FD82BD8B4D92BD8B4DA2BD8B42C
:10112000DB2B006A016A026A036ADC6BDD6BDE6B33
:10113000DF6BDB51DA11D911D8112CE0200EE06FF2
:10114000D890D437D537D637D737DC37DD37DE37C9
:10115000DF37DB51DF5D08E1DA51DE5D05E1D951B2
:10116000DD5D02E1D851DC5D0FE3D851DC5FD95180
:10117000D8A0D93DDD5FDA51D8A0DA3DDE5FDB5182
:10118000D8A0DB3DDF5FD88000360136023603365B
:10119000E02FD6D7E1AF0BD0001E011E021E031EAA
:1011A000002AD8B4012AD8B4022AD8B4032A010EDE
:1011B000EA6EDC0EE96E000105EF09F00101CF9146
:1011C00022B83AD0C45103082AE2CF81C4C100F04A
:1011D000016A026A036A03C0D3F102C0D2F101C0FE
:1011E000D1F1C4C1D0F1C3C1D7F1C2C1D6F1C1C1DF
:1011F000D5F1C0C1D4F103C0DBF102C0DAF101C006
:10120000D9F1C4C1D8F100016DD703C0C3F102C048
:10121000C2F101C0C1F100C0C0F105D00101C36B32
:10122000C26BC16BC06B010E0101E46FB70EE36FBF
:10123000000113EC05F00101186AF2BE188EF29E4F
:10124000070EF96F020EFA6F0001DFEC00F018BE16
:10125000F28E0101CFA102D0000E01D0040E186A57
:10126000F2BE188EF29EFB6F370EFC6F0001BCECD5
:1012700000F018BEF28E186AF2BE188EF29E5DEC77
:1012800001F018BEF28E22942298F5EF09F0F86A68
:10129000D09E0D8EFE0E006E060E016E020EE96EE1
:1012A000000EEA6EEE6A002EFDD7012EFBD7EA6A29
:1012B000E96A400EAF6EA60EAC6E900EAB6EC180AA
:1012C000C182C184C196196A1A6A000E926EC30E59
:1012D000936E800E946E100E956E2286010E0101A3
:1012E000D06FB70ECF6F000117EF02F001520AE185
:1012F000020E0101BB6FC36BC26BC16BC06BC56BD0
:1013000022960001D190800ED56EB50ECD6E0B0EDB
:10131000CF6EDB0ECE6E1D6A1E6A1F6A216A206ABE
:10132000229022940101C96BC86B7A0EC76F880E98
:10133000C66FCE6BCA6B2B6A2C6A0A0E2D6E2F6B92
:10134000306B316BB26B22929D809D8AC00EF2127F
:101350008C948C868C928C80FA0EE36F000154EC96
:1013600002F08C968C948C908C92FA0E0101E36FB3
:10137000000154EC02F08C948C868C928C80FA0ED6
:101380000101E36F000154EC02F08C968C948C9078
:101390008C9268EC02F001520DE0E2EF02F0015293
:1013A00009E0BFEF03F00101C96BC86BC76B7F0E8B
:1013B000C66F00010101315309E0000185EF04F01F
:1013C000015202E050EF05F00101316B22A00ED076
:1013D000229022A40BD0B52BB551130807E28C96AE
:1013E0008C948C908C920001E9D6010122A40CD03F
:1013F0001D50040805E38C948C868C908C8204D05C
:0E1400008C968C848C928C800001C3D70300E4
:020000040030CA
:00000001FF
